:100000009528A2005C200C080D04031990288A2072
:1000100084132208800664000D280E288C0A031918
:100020008D0F0B288006902825088C0023088D0052
:1000300001308E0064003620031C29288E0B1A28FC
:10004000FF308C07031C8D07031C902832308E0074
:100050001A28412008308F00422036208E0C30288C
:100060008F0B2C28422003140E080800240884005B
:100070002208841780048413000521192206FF3EFC
:1000800008002117210D06398C0050208D008C0AA4
:100090005020211F6E2821138C00023085206E28ED
:1000A00000308A000C08820701347534033415349B
:1000B00000343C340C34D934FF3A8417800590283E
:1000C0008F018E00FF308E07031C8F07031C9028C2
:1000D00003308D00DF306E2062288D01E83E8C00F9
:1000E0008D09FC30031C77288C07031874288C07B3
:1000F00064008D0F74280C187D288C1C812800004A
:100100008128080003108D0C8C0CFF3E03188228F8
:100110000C0890288C098D098C0A03198D0A080097
:1001200083130313831264000800FA306020053043
:10013000A4000230A2000430A1001E30A500A301DB
:100140001420031CCC28073C031DA0281420031CEA
:10015000CC280B3C031DA0281420031CCC28A6008F
:100160001420031CCC28A7001420031CCC28A800B2
:100170001420031CCC28A9001420031CCC28AA009E
:100180001420031CCC28AB001420031CCC28AC008A
:100190001420031CCC28AD0026088C008D010630ED
:1001A00084000130012027088C008D010630840076
:1001B0000230012028088C008D01063084000430B4
:1001C000012029088C008D010630840008300120B0
:1001D0002A088C008D0106308400103001202B0885
:1001E0008C008D0106308400203001202C088C000A
:1001F0008D0106308400403001202D088C008D01D7
:0A02000006308400803001209728AA
:02400E00F53F7C
:00000001FF
